:100000000C9462000C94FB190C94281A0C948A002E
:100010000C948A000C948A000C948A000C948A0038
:100020000C948A000C948A000C948A000C948A0028
:100030000C948A000C94370B0C948A000C948A0060
:100040000C94551A0C948A000C94D11D0C94141E17
:100050000C948A000C948A000C948A000C948A00F8
:100060000C9498080C948A0000000007000201001C
:100070000003040600000000000000000102040864
:100080001020408001020408102001020408102002
:10009000040404040404040402020202020203032E
:1000A00003030303000000002300260029000000D2
:1000B0000000250028002B0000000000240027007D
:1000C0002A00021F11241FBECFEFD8E0DEBFCDBF34
:1000D00012E0A0E0B1E0E8E7F0E402C005900D9284
:1000E000A83CB107D9F714E0A8ECB2E001C01D921A
:1000F000A23BB107E1F710E0C4ECD0E004C02297C6
:10010000FE010E941720C23CD107C9F70E943E1F82
:100110000C943A200C9400008091FA03813019F479
:1001200082E08093FA038091FA03833019F484E02B
:100130008093FA030895A8950895CF93DF93FC0167
:10014000962F9270862F817060FF20C0992331F026
:100150008091460380831092C80216C0A091C80205
:10016000C091DD03C770D0E0CC56DD4F8881A81761
:1001700010F080E03CC081E08A0F8093C802B0E0BC
:10018000AA50BD4F8C91808381E031C09923C1F08A
:1001900090819093C9021092C802292F207E2036A8
:1001A00051F490914603923020F390819F71909387
:1001B000880393E01AC09E3F39F71092460317C098
:1001C0009091C9029F3F01F79091C802993288F639
:1001D00021E0290F2093C8023081E92FF0E0EB5491
:1001E000FC4F3083293281F691E090934603DF91F2
:1001F000CF910895DC01ED91FC910190F081E02D0B
:1002000009950895DC01ED91FC910190F081E02DBC
:100210000995089560E089E00E94631B61E088E031
:100220000E94631B61E087E00E94631B60E082E044
:100230000E94631B61E084E00E94631B089542E01A
:1002400050E06CE870E080E00E94DB190895E3E084
:10025000F0E089E080935700E491E67081E0E630B9
:1002600009F080E00895CF93DF93C82F0E94270103
:10027000882381F0DFB781E08093F903F8940E942E
:100280009B0088E180936000C0936000C1110E94D0
:100290009B00DFBFDF91CF9108952091B303309190
:1002A000B403382748E0C901880F991F37FF06C0FB
:1002B0009C0151E2252750E1352701C09C014150A6
:1002C00091F73093B4032093B3030895D82FC0E07F
:1002D000CD1780F42D9A64E670E080E090E00E94F3
:1002E000CE1A2D9864E670E080E090E00E94CE1A6D
:1002F000CF5FEECF6CE271E080E090E00E94CE1A1A
:10030000E6CF0F931F93CF93DF93EC01062F15E0F9
:10031000115051F0CE010E942420081741F0602FA7
:10032000CE010E942C20F4CF82E00E946601DF9172
:10033000CF911F910F910895A0E0B0E0E2EAF1E0C3
:100340000C94E01F482E562EC0E0D0E0612C712C9A
:10035000E12CF12C00E010E0442079F081E0481617
:10036000A1F092E0491219C078E4672E712CE0E206
:10037000EE2EF12C09E413E010C0612C712CBBE1CE
:10038000EB2EF12C0EED13E008C0FDE16F2E712C69
:10039000A9E2EA2EF12C05EB13E043018C0E9D1E21
:1003A0001092B4031092B3033401A62CA818B12CF8
:1003B000C30101966C01AE14BF04A8F4A00EB11ED7
:1003C000511006C0C3010E942420F501808305C09E
:1003D000F5016081C3010E948101F50180810E94C5
:1003E0004D013601E2CFC301511018C0C3010E9474
:1003F0002420B82EC6010E9424202B2D30E0322F5D
:100400002227282B8091B3039091B403821793077E
:1004100079F4C0E0D0E0552453949ECF360160912A
:10042000B4030E9481016091B303C6010E9481015F
:10043000D395C13093E0D90708F48ECF852DCDB781
:10044000DEB7E0E10C94FC1F60E081E00E949C01BB
:10045000882331F081E09091B503973309F080E073
:10046000089561E081E00E949C0108958436910521
:1004700020F4BC0180E090E017C09C018E3B910508
:1004800028F42A553109AAE0B0E00CC0823D91055C
:1004900028F4245B3109A4E6B0E004C02D5C3109E6
:1004A000A8E5B2E00E944B1FA4E6B0E09B01AC01BE
:1004B0000E945A1F089590E08C599F4F0E94360267
:1004C000089561E082E00E949C01089560E082E06E
:1004D0000E949C01811106C08FEF9FEF90934A0309
:1004E00080934903089597E09093DE0390E2909300
:1004F000DF0391E29093E0031092E10396E2909380
:10050000E2039093E30394E29093E40395E29093E3
:10051000E50392E09093EC039FEF9093ED039AE054
:100520009093F6031092F7031092F8031092EE03E3
:100530001092EF031092F0031092F1032EE120933A
:10054000F2039093F30328EB3BE03093F503209301
:10055000F403882361F061E080E00E949C018FEF4A
:100560009FEF90934A03809349030E94610208958C
:1005700060E080E00E949C01811103C081E00E9444
:1005800073020895FC0140A5842F877090E0959533
:1005900087950196242F217030E0820F931F880FDA
:1005A000880F08958F929F92AF92BF92CF92DF9261
:1005B000EF92FF92CF93FC01C0A5EC2FE770F0E023
:1005C000EC56FD4FA081B0E0C7FF03C024E130E04E
:1005D00002C02FE030E0FC0197A183E1989FF00179
:1005E0001124E25CFE4F80809180A280B380A20F34
:1005F000B31F20E43FE14DE750E00E94651FA501D5
:1006000094010E949D1F8C2F887149F469017A0121
:10061000E0EDCE0EE7E0DE1EE11CF11C1BC0C7FFC3
:1006200005C060E47AE88CE29EE004C060E07EEE03
:100630008AEB9BE069017A01F8EBCF0EFBE0DF1E4D
:10064000E11CF11CA50194010E949D1FC20ED31E46
:10065000E41EF51EC701B60169517C4F8F4F9F4FB5
:1006600028EE33E040E050E00E949D1FA8EEB3E08A
:100670000E945A1FCF91FF90EF90DF90CF90BF90D4
:10068000AF909F908F900895DB01FA01582F5695F7
:1006900090E02481237030E0322F22274081240F04
:1006A000311D11963C932E9344814C70218130E092
:1006B00060E4469F200D311D112413963C932E9328
:1006C000129744814073228130E060E1469F200D03
:1006D000311D112415963C932E9314974481407C30
:1006E000238130E064E0469F200D311D11241796D0
:1006F0003C932E931697359618969F5F591748F698
:1007000080FF47C0408142954695469543702DE451
:1007100031E0429FC001439F900D11240C96119629
:100720009C938E93808190E044E0969587954A95BE
:10073000E1F783709927829FA001839F500D929FBC
:10074000500D1124445F5F4F13965C934E931297A4
:10075000808190E0969587959695879583709927E7
:10076000829FA001839F500D929F500D1124445FE2
:100770005F4F15965C934E93149740814370429F50
:10078000C001439F900D11240C9617969C938E9355
:1007900016970895803223E0920708F1883E23E0FF
:1007A000920740F48F519340E4E096958795EA953F
:1007B000E1F70895803D27E0920718F48C5D93409F
:1007C0000895883928E0920768F4885C974074E0BF
:1007D000969587957A95E1F78D509C4F089580E026
:1007E00090E008958FEF93E008958C30910540F4E8
:1007F000A4E0880F991FAA95E1F7885D9C4F0895A2
:10080000843F23E0920718F484529C4F0895811589
:1008100024E0920740F48657934FF4E0880F991F25
:10082000FA95E1F7089580E998E008959C013695DE
:10083000279525753575821B930B9C0123733373A4
:10084000969587959695879583739373820F931FDB
:100850009C0154E0369527955A95E1F7280F391FEA
:100860002F703F7041E051E0249FC001259F900D03
:10087000349F900D1124892F08955F98882319F0D3
:100880000000289A02C00000289800005F9A00002B
:1008900008955F9A000083B15F980000869581708B
:1008A0000895CF93DF93D82F5C9A5F985C98C8E047
:1008B0008D2F80780E943D04DD0FC150C9F75F98ED
:1008C000DF91CF9108958F770E9451040895CF93BF
:1008D000DF93D82FC8E08D2F80780E943D04DD0F74
:1008E000C150C9F75F98DF91CF910895CF93DF93FF
:1008F0005F98C8E080E0D82FDD0F0E9449048D0F7B
:10090000C150C9F7DF91CF9108950E9463040E94FE
:1009100076045C9A0895A1E0B0E0E1E9F4E00C947B
:10092000EE1F806869830E9451046981862F0E94AE
:1009300067045C9A2196E2E00C940A20CF93C09160
:10094000BE03C827E82FF0E0EB54FC4F678589E72A
:100950000E948B046C2F8DE30E948B046C2F82E429
:100960000E948B04CF91089586E20E948504089529
:10097000CF938BE20E948504C82F8CE20E948504ED
:10098000282F30E066E0369527956A95E1F744E038
:10099000C49FC0011124822B932BCF910895CF9334
:1009A000DF93EC016C818CE10E948B046D818DE101
:1009B0000E948B046E818EE10E948B046F8180E225
:1009C0000E948B04688581E20E948B04698582E223
:1009D0000E948B046A8583E20E948B046B8584E20B
:1009E0000E948B046C8585E20E948B046D858AE2EF
:1009F0000E948B046E858EE60E948B046F858FE6C5
:100A00000E948B04688980E70E948B04698981E7D2
:100A10000E948B046A8982E70E948B04DF91CF9148
:100A20000895CF92DF92EF92FF92CF93DF936B0105
:100A30007C01C11488E3D8068CE9E8068CE1F8064D
:100A400028F5C701B60120E836E948E950E00E94E0
:100A50009D1FE901689760E879E687E69FEF0E94AD
:100A60006D1F6C0D7D1D8E1D9F1DF2E0660F771FA3
:100A7000881F991FFA95D1F721E732E040E050E056
:100A80000E949D1FF22EE32E80E421C0C701B60113
:100A900020E03DE241E351E00E949D1FE90168979B
:100AA00060E073ED8EEC9EEF0E946D1F6C0D7D1D5E
:100AB0008E1D9F1D660F771F881F991F21E732E04B
:100AC00040E050E00E949D1FF22EE32E80E66C2F46
:100AD0006F71680F85E70E948B046E2D86E70E9478
:100AE0008B046F2D87E70E948B04DF91CF91FF90DD
:100AF000EF90DF90CF9008958F929F92AF92BF9228
:100B0000CF92DF92EF92FF92CF93DF93D82F83E0C3
:100B10000E9485048093B20384E00E948504809340
:100B2000B10360E086E00E948B0461E087E00E94F0
:100B30008B046FE789E00E948B0465E08AE00E94E5
:100B40008B0462E18BE00E948B0465E18CE00E94E3
:100B50008B046DEF8DE00E948B0460E08EE00E94BC
:100B60008B04DD2319F08BE291E008C02091DC03B7
:100B700033E1239FC0011124825C9E4F0E94CF0469
:100B80006CE880E30E948B046FE082E30E948B0498
:100B900062E483E30E948B048091DD0387FF02C03F
:100BA00064E101C06AE084E30E948B046AE285E3A9
:100BB0000E948B046DE286E30E948B0464ED87E360
:100BC0000E948B0460E088E30E948B0460E089E36C
:100BD0000E948B04D11109C0C090BE03D090BF0306
:100BE000E090C003F090C10307C0C5E8CC2EC1EC73
:100BF000DC2EED2CCEEDFC2ECAE38F2C9924AA24FA
:100C0000BB24682D8C2F0E948B04682D85E08C0FEF
:100C10000E948B04FE2CED2CDC2CCC24CF5FCE3339
:100C200061F76FEF83E40E948B046FEF84E40E940E
:100C30008B046FEF85E40E948B046FEF86E40E94C3
:100C40008B04DD2311F066E002C06091C2038DE6E3
:100C50000E948B0460E089E70E948B046091C303CB
:100C60008AE70E948B0460E083E70E948B0460E0C7
:100C700084E70E948B04D11109C06091BA0370917E
:100C8000BB038091BC039091BD0304C060EC7AEC7F
:100C900089E896E30E941105DF91CF91FF90EF90D4
:100CA000DF90CF90BF90AF909F908F90089561E0BC
:100CB00087E00E948B0464E28EE70E948B0463E06D
:100CC00088E00E948B0460E088E00E948B0465E06D
:100CD00087E00E948B0462E085E00E948B0483E041
:100CE0000E9485048093B20384E00E94850480936F
:100CF000B103089583E00E9485048093B20384E0E9
:100D00000E9485048093B10361E087E00E948B0418
:100D10006AE070E080E090E00E94CE1A0E945706E0
:100D200000000895CF92DF92FF920F931F93CF930D
:100D3000DF931F92CDB7DEB7082F162F8EE399836E
:100D40000E948B04F02EC02E9981D92E8C2D8F19E4
:100D5000811738F4F60161916F018FE70E948B04CF
:100D6000F5CF64E085E00E948B0483E00E94850457
:100D70008093B20384E00E9485048093B1030E94B3
:100D8000AB1A6093AD037093AE038093AF0390935F
:100D9000B00369E087E00E948B0481E08093FA034E
:100DA0000F90DF91CF911F910F91FF90DF90CF9027
:100DB00008950F931F930E9492068091FA03813049
:100DC00099F40E94AB1A0091AD031091AE032091EB
:100DD000AF033091B003601B710B820B930B603A31
:100DE00076488140910548F38091FA03813031F4CF
:100DF00068EB71E088E094E00E946D1C1F910F91F8
:100E000008950F931F938091FA03823021F410927A
:100E1000FA0381E020C08091FA038130D9F40E9466
:100E2000AB1A0091AD031091AE032091AF03309146
:100E3000B003601B710B820B930B613A76488140C3
:100E4000910540F061E087E00E948B041092FA0364
:100E500082E001C080E01F910F910895EF92FF9210
:100E60000F931F93CF93DF938B019C01442737FD92
:100E70004095542F60E271EA87E090E00E94BF1F26
:100E8000E9011C161D0614F0C1E0D0E0D80120E2F3
:100E900031EA47E050E00E94651F9E01442737FD7C
:100EA0004095542F0E94BF1F790100E010E00E15FD
:100EB0001F055CF4289ACE010E94F41A2898CE01EE
:100EC0000E94F41A0F5F1F4FF2CFCDB7DEB7E6E0F6
:100ED0000C940620CF93C82F2C9A83E00E9485049F
:100EE0008093B20384E00E9485048093B10360E0A4
:100EF00086E00E948B0461E087E00E948B046FE72C
:100F000089E00E948B0465E08AE00E948B0462E124
:100F10008BE00E948B0465E18CE00E948B046DEFF6
:100F20008DE00E948B0460E08EE00E948B046CE2F6
:100F300080E70E948B0460E080E30E948B0460E005
:100F400089E70E948B0465E08AE70E948B0462E1D6
:100F500081E70E948B0462E082E70E948B0460E0DC
:100F600083E70E948B0460E084E70E948B04609119
:100F7000EE037091EF038091F0039091F1030E94D2
:100F8000110567E08DE60E948B046AE070E080E066
:100F900090E00E94CE1A69E087E00E948B046AE02C
:100FA00070E080E090E00E94CE1ACC2369F0C5E1A9
:100FB000C15009F459C061E070E088EB91E00E94F3
:100FC0002E070E949B00F4CF61E070E088E891E07A
:100FD0000E942E070E949B0065E08DE60E948B0414
:100FE0006AE070E080E090E00E94CE1A61E070E07C
:100FF00088EB91E00E942E070E949B0064E08DE642
:101000000E948B046AE070E080E090E00E94CE1ABB
:1010100061E070E08DE591E00E942E070E949B0048
:1010200062E08DE60E948B046AE070E080E090E070
:101030000E94CE1A61E070E08FEA90E00E942E07D5
:101040000E949B0060E08DE60E948B046AE070E0E5
:1010500080E090E00E94CE1A62E070E085E091E0CE
:101060000E942E070E949B0061E087E00E948B0493
:101070002C98CF910895CF93DF93EC014AE050E094
:101080006D2F70E088E094E00E94321D6EE288E0EF
:1010900094E00E94511CBE0184E0769567958A9584
:1010A000E1F76F7077274AE050E088E094E00E9413
:1010B000321D6EE288E094E00E94511CBE016F7008
:1010C00077274AE050E088E094E00E94321DDF91EB
:1010D000CF910895CF93C1E0811101C0C0E06C2F82
:1010E00082E10E949C1B6C2F83E10E949C1B10924A
:1010F000A7031092A6038091B9008C6F8093B9006A
:1011000080E28093B80085E48093BC00CF9108957D
:1011100085ED8093BC008091BC0084FDFCCF0895D8
:10112000ECEBF0E0108285E480831092A603089532
:101130001F920F920FB60F9211242F933F934F934C
:101140005F936F937F938F939F93AF93BF93EF932F
:10115000FF93CF93DF931F92CDB7DEB78091B90095
:10116000887F803609F4C7C0A8F5883209F464C0C6
:1011700098F4803109F45DC038F4882309F4F3C091
:10118000883009F456C0F1C0883109F455C0803266
:1011900009F0EBC082E0A7C0803409F477C078F48E
:1011A000803309F45FC0883309F0DFC084E08093A6
:1011B000A5038091A6038B7F8093A603D0C08035C2
:1011C00009F452C0883509F467C0883409F0CDC0ED
:1011D00085E089C0883909F4C0C0A8F4883709F4CB
:1011E0008AC038F4883609F486C0803709F483C091
:1011F000BCC0883809F4B1C0803909F47FC0803898
:1012000009F0B3C07BC0803B09F493C038F4803A46
:1012100009F48CC0883A09F48CC0A7C0803C09F45A
:101220009EC0883C09F49BC0883B09F09EC080E0CA
:1012300081C08091AA0313C08091A7039FEF980FEC
:101240009093A7038823D1F1E091A803F091A9031B
:10125000CF0101969093A9038093A8038081809386
:10126000BB007DC083E03FC0E091A803F091A903DB
:10127000CF0101969093A9038093A8038091BB00AE
:1012800080838091A70381508093A7038091A70357
:10129000823008F064C061C0E091A803F091A90316
:1012A000CF0101969093A9038093A8038091BB007E
:1012B00080838091A70381508093A7038091A60328
:1012C0008B7F8093A6038091A60380FF4CC0809102
:1012D000A6038E7F8093A6038091A60382608093ED
:1012E000A60384EA3DC08093A5038091A6038B7F6B
:1012F0008093A60338C01092A70331C0E091AB03DE
:10130000F091AC03309749F18091BB0089838091C3
:10131000A70391E0980F9093A703811102C062E0A8
:1013200001C060E0CE010196099515C00E948808B1
:1013300016C081E0E091AB03F091AC03309769F007
:10134000882311F063E001C061E0CE0101960995A8
:1013500099819093BB00811102C085E801C085ECA2
:101360008093BC0002C00E9488080F90DF91CF914B
:10137000FF91EF91BF91AF919F918F917F916F916D
:101380005F914F913F912F910F900FBE0F901F9043
:1013900018958F929F92AF92BF92CF92DF92EF9269
:1013A000FF92CF93DF93EC010E94AB1A6B017C019B
:1013B0004E01A12CB12C8091A60382FF11C0209771
:1013C000D1F30E94AB1A6C197D098E099F0986160C
:1013D0009706A806B90678F70E94900881E004C035
:1013E0008091A5031092A503DF91CF91FF90EF901C
:1013F000DF90CF90BF90AF909F908F900895A2E024
:10140000B0E0E5E0FAE00C94EA1F182F7B01022F10
:10141000047022FD05C08091090190910A0102C06B
:1014200080E090E02A8349830E94C9092A8149818A
:10143000811136C01092A5034093A703F092A9032F
:10144000E092A803110F1093AA039091A60321FF25
:1014500002C085E001C084E0892B8093A6038091BF
:10146000A60381FF0BC08091A6038D7F8093A60306
:101470008091AA038093BB0085EC01C085EE809328
:10148000BC00822F817020FF0BC0011105C080912C
:10149000090190910A0102C080E090E00E94C90910
:1014A0002296E6E00C940620A2E0B0E0EAE5FAE03D
:1014B0000C94EA1F182F7B01022F047022FD05C037
:1014C0008091090190910A0102C080E090E02A8396
:1014D00049830E94C9092A814981811138C010922B
:1014E000A5034093A703F092A903E092A803812FDC
:1014F000880F81608093AA039091A60321FF02C008
:1015000085E001C084E0892B8093A6038091A60327
:1015100081FF0BC08091A6038D7F8093A6038091ED
:10152000AA038093BB0085EC01C085EE8093BC00CC
:10153000822F817020FF0BC0011105C0809109012D
:1015400090910A0102C080E090E00E94C9092296B1
:10155000E6E00C940620A0E0B0E0E1EBFAE00C94A9
:10156000E81F0E94AB1A0091A1031091A2032091E1
:10157000A3033091A4036B017C01C01AD10AE20AD3
:10158000F30A9701860141E1C41647E2D406E1045B
:10159000F10408F442C02091A00331E0320F3093EF
:1015A000A00320FF02C017E001C010E06093A10378
:1015B0007093A2038093A3039093A40363E070E06D
:1015C00088E094E00E94020161E070E088E094E02D
:1015D0000E94020107E0010F812F90E0EC01CC0F87
:1015E000DD1FC55FDE4F68817981672F77276370C4
:1015F0007727880F991F880F991F682B792B88E010
:1016000094E00E94FA0068817981772788E094E06D
:101610000E94FA001F5F1013DFCFCDB7DEB7E8E0FE
:101620000C94042025B190E0FC01EE0FFF1FE80FA1
:10163000F91FE05FFC4F8081282B25B988B191818B
:10164000892B88B98BB19281892B8BB9089585B18B
:1016500090910D03892385B988B190910E03892358
:1016600088B98BB190910F0389238BB908951F928C
:101670000F920FB60F9211242F933F934F935F93C6
:101680006F937F938F939F93AF93BF93CF93EF937A
:10169000FF93C0916C0380910601C81708F03EC00B
:1016A00080910B0390910C039093870080938600A8
:1016B000EC2FF0E0EE0FFF1FE55FFE4F8081918180
:1016C0000E94F503880F991F90930C0380930B03DE
:1016D00080910B0390910C03209107013091080138
:1016E000281B390B30930801209307018091F403E4
:1016F0009091F503880F991F2817390720F49093CC
:1017000008018093070180916A03811142C0809192
:10171000EC0380FF41C0C830E0F53EC080910B0370
:1017200090910C039093870080938600809107012D
:101730009091080190930C0380930B0380916A03AE
:10174000882319F08FEF9FEF06C080910B039091D3
:101750000C038855924090938B0080938A0080E41C
:101760009CE99093080180930701809184009091F7
:1017700085008097D0F30E94270B80916B03811125
:1017800005C08091060181500E94120B10926C03DB
:1017900027C08FEF9FEF06C080910B0390910C0341
:1017A0008855924090938B0080938A0080918400AA
:1017B000909185008097D0F30E94270B80916B0356
:1017C000811104C080916C03811106C080916C036B
:1017D0008F5F80936C0304C081500E94120BF6CF80
:1017E000FF91EF91CF91BF91AF919F918F917F9199
:1017F0006F915F914F913F912F910F900FBE0F907E
:101800001F90189524E0829FC00111248C3091050F
:1018100038F0853F23E0920728F084EF93E00895A5
:101820008CE090E00895CF93DF93C091ED03C03337
:1018300090F48C2F807339F0803141F480916D03E6
:101840008295807F05C08091720302C080917303EE
:10185000CF70D0E015C0CF33E0F4CF70D0E08091EE
:101860006D038295807F0E94020CDE01AA0FBB1FD0
:10187000A55FBE4F11969C938E9321968091730322
:101880000E94020CFE01EE0FFF1FE55FFE4F9183E9
:101890008083DF91CF91089580916E0390916F03C3
:1018A0009F770E94160480936D038F3029F48091F6
:1018B00073038695805804C099E0899F802D112478
:1018C00080937203F8940E94130C78948091E00343
:1018D0008132E1F4809172039FEF980F9E3F78F080
:1018E0008091B0008F7D8093B00061E080917203A1
:1018F000811101C060E083E00E949C1B08958093E9
:10190000B4008091B00080628093B0000895FF928F
:101910000F931F93CF93DF930FED13E0C0E0D0E060
:10192000B3E0FB2E8C2FD801ED918D019E2F907F7F
:101930009031F1F4EF70F0E0EE0FFF1FE55FFE4F26
:10194000208131816F2D0E947D1FE92FF0E0EE0F85
:10195000FF1FE257FD4F61E080819181821793075D
:1019600008F060E0FE01E456FD4F80810E949C1B60
:101970002196C730D105B1F6CDB7DEB7E5E00C94BE
:1019800007208091490390914A03019631F1E9E4DF
:10199000F3E080E090E04091ED03242F2F7030E0E1
:1019A0008217930799F02F5F3F4F8217930711F427
:1019B000403360F4F89420813181DC01AA0FBB1F11
:1019C000A55FBE4F11963C932E9378940196329664
:1019D0008031910501F70E94870C0895FF920F93C3
:1019E0001F93CF93DF9385EB93E00E94C202809315
:1019F00006019091ED03292F2F70281304C081E078
:101A0000820F8093060190539F3060F4409106014D
:101A100030E0842F90E001972817390719F44F5FC1
:101A20004093060180910601813118F080E1809396
:101A30000601E2E1F3E0DF0112971C92DF0111974A
:101A40001C921082339623E0E732F207A1F74FEFA2
:101A50003FEFA5EAB2E00FED13E02FEFE801899127
:101A60008E018031F8F490E0FD0132976081FC0135
:101A7000EE0FFF1FE80FF91FE05FFC4F8081862B00
:101A80008083CD010197EC0158818181852B818371
:101A90009C918281892B8283609550959095292312
:101AA000352346231396D3E0063E1D07B9F640932F
:101AB0000D0330930E0320930F03CCE9D2E00FED1A
:101AC00013E0F12CF80181918F01823230F08632DF
:101AD000B8F0863211F460E010C0F5E0FF1204C0E7
:101AE0008091C1008F7E06C026E0F21205C0809171
:101AF000C100877F8093C10061E088810E94631BE1
:101B0000F394219687E0F812DDCF8091DF038032D5
:101B100031F461E08AE00E949C1B82E201C082E015
:101B20008093800081E080936B0380936A038091AF
:101B3000E003813211F08732D9F461E083E00E9442
:101B4000631B60E083E00E949C1B8091E003813274
:101B500031F481E08093B0008093B10009C082E04D
:101B60008093B00085E08093B1008EE38093B30052
:101B70008AE1809381008FEF9FEF90938B00809399
:101B80008A0080ED97E0909387008093860080E440
:101B90009CE9909308018093070190930C03809334
:101BA0000B0310926C0380916F00816080936F0033
:101BB0008091EC0383FF0CC08091490390914A030C
:101BC000019631F00E94C10C10926A0310926B03CF
:101BD000CDB7DEB7E5E00C940720CF93C82F8091F6
:101BE000E1038B3221F46C2F8EE00E949C1B8091CC
:101BF000E003873249F48091B000CC2311F080617A
:101C000001C08F7E8093B000CF910895A3E2B0E031
:101C1000ECE0FEE00C94DE1F6B017C010E949F1A39
:101C20004B015C0181E00E947C0583E08093FA0314
:101C30000E947A0664EC71E088E094E00E946D1CDA
:101C400044244A94542CF6E42F2EA5E53A2EC114D0
:101C5000D104E104F10469F00E949F1A681979091E
:101C60008A099B096C157D058E059F0510F080E0A3
:101C7000E5C08091FA03843051F762ED71E088E0AD
:101C800094E00E946D1C8FE70E9463040E9476041A
:101C90008AA3823601F505EB13E00E947604F80171
:101CA00081938F01F3E00E3D1F07B9F78091B503D3
:101CB000873309F0BDC06BED71E088E094E00E94CD
:101CC0006D1C82E48AA361E0CE0182960E94D9064F
:101CD0002C9A81E0B3C0803741F0893619F581E054
:101CE0000E94730289E4898305C020E52983C12C01
:101CF000D12C76019091F9038091EC03992311F096
:101D0000806801C08F778093EC03EEEDF3E0DE0195
:101D100012968BE101900D928A95E1F76CE1CE016C
:101D2000019684C08437D9F494E5998393E09A832B
:101D30008B8387E08C838DE08D838AE1EDE9F1E090
:101D4000DE01169601900D928A95E1F76FE1CE01C2
:101D500001960E94D906C12CD12C760169C0853725
:101D600089F40EED13E00E947604F80181938F014F
:101D7000F3E0093F1F07B9F761E080E00E949C0192
:101D80003AA251C0863629F52091490330914A0381
:101D90002F3F3F4FD9F0298279E4672E73E0772EE9
:101DA0008E010D5F1F4FF301819191913F010E94C0
:101DB000F503F80131979083F80180830E5F1F4F80
:101DC000F9E66F16F3E07F0671F701C0898361E2DF
:101DD000A6CF8736E9F409E413E00E947604682E62
:101DE000712C762C66240E9476049301280F311DF5
:101DF000C9010E94CA03F801819391938F01F3E016
:101E000009361F0751F727E42AA30E9461020BC07D
:101E1000873471F450924A03409249038BA30E9485
:101E200061028BA18AA361E0CE0182960E94D9064D
:101E300083E08093FA030E94570609CFA396E2E15C
:101E40000C94FA1F1F93CF93DF93C82FD62F61E016
:101E50000E94631B61E08C2F0E949C1B61E08D2F10
:101E60000E949C1B8AE090E00E94F41A8D2F0E9431
:101E7000CF1B892B71F060E08C2F0E949C1B8AE0A5
:101E800090E00E94F41A8D2F0E94CF1B11E0892B45
:101E900009F010E060E08C2F0E94631B60E08C2F43
:101EA0000E949C1B60E08D2F0E949C1B812FDF9164
:101EB000CF911F91089580E48093BA001092BD00E5
:101EC0008DE990E09093AC038093AB0310924603AE
:101ED00015E004E0B2E0FB2E80914603813039F436
:101EE00080E00E947C05F09246032D98F5CFC091CA
:101EF0004603C33061F42C98809188030E949E04AD
:101F0000C093FA030E94570600934603E5CF8091E1
:101F10004603843009F78091FA038430E9F68FE7AD
:101F20000E946304C6EFD2E0E091DD03E770F0E0C9
:101F3000EC56FD4F808190E09E01265F32402817CD
:101F4000390724F40E9476048993EECF1093460358
:101F50002C9AC2CFAAE2B0E0E0EBFFE00C94ED1FB8
:101F60001FEF198389E2E5EBF3E0DE0112960190A1
:101F70000D928A95E1F721E04AE2BE016F5F7F4F43
:101F800080E20E94FF0981110EC021E041E0BE0104
:101F90006F5F7F4F80E20E94540A811104C082E08B
:101FA0008093460302C0109346038091460382301B
:101FB00051F00E949F1A60934203709343038093F1
:101FC000440390934503AA96E3E00C940920A1E012
:101FD000B0E0EDEEFFE00C94EE1F809146038230FE
:101FE000D9F480918803805A898321E041E0BE01C1
:101FF0006F5F7F4F80E20E94FF09882369F08FEFB7
:10200000809346030E949F1A609342037093430398
:1020100080934403909345032196E2E00C940A20B8
:10202000A1E0B0E0E6E1F0E10C94EE1F8091460300
:102030008230D1F421E041E0BE016F5F7F4F80E24A
:102040000E94540A882371F08FEF809346030E9408
:102050009F1A6093420370934303809344039093C9
:10206000450302C0898101C08FEF2196E2E00C9404
:102070000A20A2E2B0E0EFE3F0E10C94DE1F9E0143
:102080002F5F3F4F80E1D9011D928A95E9F766EEF7
:1020900071E088E094E029A33AA30E946D1C0E949D
:1020A0007A061D8A1E8A1F8A188E312C212C00E088
:1020B000812C912C540180EC482E8DE9582E88E516
:1020C000682E85E3782E90E5C92E93ECD92EE12C6D
:1020D000F12C84EF91E0A0E0B0E08D8F9E8FAF8F68
:1020E000B8A380EC97EFAAEBB7E3898F9A8FAB8FF9
:1020F000BC8F80EC9DE9A8E5B5E3898B9A8BAB8B0F
:10210000BC8B88E094E00E94391D892B09F4E1C062
:1021100088E094E00E94661D9C0133272C32310533
:1021200009F442C0ACF42332310509F0ABC0198286
:102130001A821B821C821D821E821F8218861986AB
:102140001A861B861C861D861E861F86188A60C0FE
:102150002434310529F02335310509F4B2C092C089
:1021600064E488E094E00E94511C2AE030E040ECF6
:102170005DE968E575E388E094E00E94CD1C6CE2BF
:1021800088E094E00E94511C2AE030E040EC57EFD8
:102190006AEB77E388E094E00E94CD1C6CE288E073
:1021A00094E00E947F1CADCF0F5F043009F0A9CFEF
:1021B00029813A814B815C81A8EEB3E00E945A1FCD
:1021C000698B7A8B8B8B9C8B2D813E814F815885BF
:1021D0000E945A1F698F7A8F8B8F9C8F29853A8531
:1021E0004B855C852D8F3E8F4F8F58A32D853E8567
:1021F0004F8558890E945A1F6B017C0160323EE472
:1022000073078105910530F462E38CE10E948B0431
:1022100000E077CF603345E774078105910510F43E
:1022200062E2F3CF60345CE975078105910510F433
:1022300066E2EBCF80E5C81683ECD806E104F10432
:1022400010F462E1E2CF90E6C9169AEED906E104F5
:10225000F10410F465E1D9CFA0E7CA16A1E1DA06CE
:10226000A1E0EA06F10410F461E0CFCFB0EACB16AA
:10227000B6E8DB06B1E0EB06F10410F463E0C5CF8D
:1022800065E0C3CF10ED180F1A3008F03ACFE1E047
:10229000F0E0EC0FFD1F24E0029FE00DF11D112482
:1022A0002081318142815381AAE0B0E00E945A1F0F
:1022B000610F711D811D911D6083718382839383E2
:1022C00020CF49885A886B887C88812C912C5401B6
:1022D00018CF81149104A104B10489F4C301B2019F
:1022E0000E94110561E070E080E090E00E94CE1A4B
:1022F0001D8A1E8A1F8A188E312C22242A948D8DC5
:102300009E8DAF8DB8A188169906AA06BB06D0F49B
:102310000E94B4042D893E894F89588D280F311DA4
:10232000411D511D2D8B3E8B4F8B588F381608F455
:10233000382E821508F4282E3FEF831A930AA30A39
:10234000B30A56C0C301B20128EE33E040E050E0CA
:102350000E949D1FBA01A9012AE030E088E094E0C4
:102360000E941B1D6CE288E094E00E94511C4AE030
:1023700050E0632D88E094E00E942A1D6CE288E022
:1023800094E00E94511C6D897E898F89988DA501EA
:1023900094010E949D1FBA01A9012AE030E088E063
:1023A00094E00E941B1D6CE288E094E00E94511CA6
:1023B0004AE050E0622D88E094E00E942A1D6CE221
:1023C00088E094E00E947F1C4C0C5D1C6E1C7F1CFE
:1023D000898D9A8DAB8DBC8D84159505A605B705A5
:1023E00020F449885A886B887C88812C912C540170
:1023F00029893A894B895C89283E3340410551053A
:1024000009F07FCEA296E2E10C94FA1FA1E0B0E0C1
:10241000ECE0F2E10C94EE1F80E00E94330161E0F9
:102420008CE00E94631B61E08DE00E94631B0E94B0
:102430000A0160E080E00E94631B61E081E00E948D
:10244000631B40E052EC61E070E088E094E00E94A1
:10245000811E0E94B8020E94660263EF71E088E06C
:1024600094E00E944E1C84E793E00E943B086AE0DF
:1024700072E088E094E00E944E1C4AE050E062E086
:1024800070E088E094E00E94031D0E941F01789490
:102490002D9A62E18EE00E94220F882329F02D9868
:1024A0002C980E943910FBCF63E08AE00E94220F33
:1024B000811104C00E942402811119C06DE472E0F0
:1024C00088E094E00E944E1C60E070E0CB010E9426
:1024D000060E882349F00E94310262E172E088E032
:1024E00094E00E946D1C2C9A0E94EE0C10C00E9479
:1024F000EE0C8091E203823209F0CAC08091E303BE
:10250000833209F0C5C08091EC0381FDC7C0809182
:10251000E203823231F58091E303833211F581E0E9
:102520000E946A088091EC0382FF08C06DE272E0AD
:1025300088E094E00E946D1C0E945B0F64E170E0F3
:1025400080E090E00E94CE1A21E041E0BE016F5F82
:102550007F4F80E20E94540A811103C081E0809382
:10256000460368E372E088E094E00E944E1C8FE02E
:102570000E94330180E00E947C051092880380E075
:102580000E949E0480E0883170F08093CA0283E04C
:102590008093FA030E947A0680914603882371F0A3
:1025A0000E94AA0F0BC021E0280FE82FF0E0EB54A7
:1025B000FC4F9785992349F3822FE5CF8091E5035E
:1025C000982F9D7F983229F440E052EC61E070E052
:1025D00027C0893271F440EA56E861E070E088E093
:1025E00094E00E94811E8091C20080628093C200AC
:1025F0001BC08091DD038871803129F440E855E2E9
:1026000060E070E00DC04091B6035091B703609157
:10261000B8037091B9034A3051056105710570F333
:1026200088E094E00E94811E88E094E00E94391DB9
:10263000892B29F088E094E00E94661DF5CF8091F7
:10264000E403843229F08091C1008F7E8093C10021
:102650008091E503853241F08852833028F08091E3
:10266000C100877F8093C1001092CC021092CB02F0
:10267000109248030E94AB1A609384037093850301
:1026800080938603909387032196E2E00C940A20BE
:102690008091EC038B7F8093EC0335CF82FD37CFA5
:1026A00064EF71E080E090E00E94060E882309F458
:1026B0002ECF0E94310262E172E088E094E00E9435
:1026C0006D1C0E94EE0C2C9A22CFCF93DF9388E0F2
:1026D00094E00E94391D892BE9F0C091CB02D0E033
:1026E000CE0101968F7199272091CC0230E082179C
:1026F000930781F088E094E00E94661DC353DD4F8C
:1027000088838091CB0290E001968F719927809306
:10271000CB02DDCFDF91CF910895A0E0B0E0E3E9F7
:10272000F3E10C94E81FD82FC62F0E94AB1A00913A
:10273000A1031091A2032091A3033091A4036B0184
:102740007C01C01AD10AE20AF30A9701860141E12D
:10275000C41647E2D406E104F10408F4D1C1609341
:10276000A1037093A2038093A3039093A403809189
:102770000B0190910C01880F991F80938903892F79
:10278000877020918A03287F282B20938A038091C9
:102790000D0190910E01880F991F382F330F330FC1
:1027A000330F2770232B20938A03282F22952695F9
:1027B000277080918B03807C9770990F990F990FE8
:1027C000822B892B80938B0320910F013091100174
:1027D000220F331F922F9295990F990F907C8F7330
:1027E000892B80938B03932F9295990F990F907C4F
:1027F000822F86958695892B80938C0332FB8827C0
:1028000080F920918D032E7F282B20938D038091BA
:10281000110190911201880F991F382F330F2170E9
:10282000232B20938D03382F331F3327331F209101
:102830008E03207F892F8770880F232B282B2093CE
:102840008E038091130190911401880F991F382FE6
:102850003295307F2F70232B20938E03382F3295A3
:102860003F7020918F032078892F87708295807F19
:10287000232B282B20938F03809115019091160113
:10288000880F991F2F7720938F03292F27952227B1
:1028900027958695822B80939003892F8695837048
:1028A000209191032C7F282B209391038091170175
:1028B00090911801880F991F382F330F330F237011
:1028C000232B20939103382F32953695369533700C
:1028D00020919203207E892F8770880F880F232BE9
:1028E000282B209392038091190190911A01880F4F
:1028F000991F382F3295330F307E2F71232B209361
:1029000092039295990F907E869586958695892B50
:102910008093930380911B0190911C01880F991F54
:1029200080939403892F877020919503287F282B0B
:102930002093950380911D0190911E01880F991F8E
:10294000382F330F330F330F2770232B209395032A
:10295000282F22952695277080919603807C97706A
:10296000990F990F990F822B892B809396032091B1
:102970001F0130912001220F331F922F9295990F42
:10298000990F907C8F73892B80939603932F929548
:10299000990F990F907C822F86958695892B80932D
:1029A000970332FB882780F9209198032E7F282BEC
:1029B000209398038091210190912201880F991F03
:1029C000382F330F2170232B20939803382F331F78
:1029D0003327331F20919903207F892F8770880F19
:1029E000232B282B2093990380912301909124017C
:1029F000880F991F382F3295307F2F70232B20930B
:102A00009903382F32953F7020919A032078892FAF
:102A100087708295807F232B282B20939A038091A7
:102A2000250190912601880F991F2F7720939A03F3
:102A3000292F2795222727958695822B80939B0304
:102A40009695937080919C038C7F892B80939C0337
:102A50002091270130912801220F331F922F990FC7
:102A6000990F8370892B80939C0322952695269538
:102A7000237080919D03807E932F9770990F990FFB
:102A8000822B892B80939D032091290130912A016B
:102A9000220F331F922F9295990F907E8F71892B61
:102AA00080939D03832F8295880F807E269526959F
:102AB0002695282B20939E03DD2311F088E001C08A
:102AC00080E0CC2311F094E001C090E0892B80934A
:102AD0009F036FE070E088E094E00E940201C9E883
:102AE000D3E0699188E094E00E94931D83E0C03AAE
:102AF000D807B9F760E070E088E094E00E94020136
:102B0000CDB7DEB7E8E00C940420CF93C82F682F30
:102B100088E094E00E94931D8C2F0E944D01CF917C
:102B20000895A0E0B0E0E7E9F5E10C94E81FC82FB4
:102B30000E94AB1A0091A1031091A2032091A3035C
:102B40003091A4036B017C01C01AD10AE20AF30A96
:102B50009701860141E1C41647E2D406E104F1047D
:102B600008F445C06093A1037093A2038093A3036C
:102B70009093A4031092B4031092B30388EA0E94C6
:102B80008515CC2311F081E801C081E00E948515F4
:102B900080E10E94851500E010E0F801EE0FFF1FB4
:102BA000E55FFE4F808191810E94F503EC01B3E067
:102BB000CC0FDD1FBA95E1F78D2F0E9485158C2F64
:102BC0000E9485150F5F1F4F0031110531F760918D
:102BD000B40370E088E094E00E94FA006091B303CF
:102BE0007091B403772788E094E00E94FA00CDB793
:102BF000DEB7E8E00C940420AAE1B0E0E2E0F6E100
:102C00000C94E01F0E949B008CE00E9485048111BF
:102C10000BC066E872E088E094E00E946D1C80E0E2
:102C20000E947C050E947A060E9465130E94AB1ADE
:102C30000E94101091E0853009F090E01FEF809124
:102C4000FA03843009F494C1911192C16EC00E94BC
:102C5000B80490937103809370032C9AC0928403FC
:102C6000D0928503E0928603F09287031092470387
:102C700080916E0390916F03880F991F81609093EC
:102C80006F0380936E032D9880E00E94ED0D80917C
:102C9000F602982F9E7309F0C2C1F8948091DD036B
:102CA00047EF52E06BE071E087700E9444030E949E
:102CB000130C78949091F6028091400390FFA9C183
:102CC000811116C0A9E4B3E080E090E0FC01EE0FB2
:102CD000FF1FE55FFE4F208131812D933D930196CB
:102CE0008031910599F70E94610281E08093400351
:102CF00080914803811103C081E0809348031092C2
:102D0000690310926B0310926A038091DD0388714E
:102D100009F0ADC10E94870C83E08093FA030E9402
:102D2000570681E0809341032C980E94AB1A4B0117
:102D30005C010E949F1A6B017C01809147038230E5
:102D400008F063C040908403509085036090860330
:102D5000709087038091800390918103A0918203FA
:102D6000B091830384159505A605B70509F44DC0F8
:102D700085EB93E00E94D2026C5D75408109910958
:102D8000950184010419150926093709601771078F
:102D900082079307D0F5409280035092810360929E
:102DA0008203709283030E94B404282F80937403DB
:102DB0008091750390917603820F911D9093760315
:102DC00080937503609177036F5F60937703693039
:102DD000E0F070E00E94891F7093760360937503A2
:102DE00080917303B3E08B9F600D711D1124769564
:102DF000679576956795609373030E944C0C1092CB
:102E00007603109275031092770380914803009126
:102E1000CA02882351F110914703101708F0CDC161
:102E200040908403509085036090860370908703E0
:102E3000A501940124193509460957092F8B388FAC
:102E4000498F5A8F85EB93E00E94D20268517C4FE4
:102E50008F4F9F4F2F89388D498D5A8D6217730779
:102E60008407950708F470C1A8C1809184039091EC
:102E70008503A0918603B091870375016401C81A88
:102E8000D90AEA0AFB0A85EB93E00E94D2029B0171
:102E9000AC01A02FB0E00E945A1F6C157D058E0575
:102EA0009F0558F48092840390928503A092860334
:102EB000B092870381E08093410380916A0381117E
:102EC00016C08091E503883219F40E94AB0A0FC046
:102ED000893239F460914703809169030E948D1310
:102EE00006C08A3221F4809169030E949115809175
:102EF00041038823B9F0E0918803EF5FE0938803F2
:102F0000E83131F0F0E0EB54FC4F8785811102C0CD
:102F100010928803809188030E949E040E94E70F0C
:102F200010924103809146038F3F09F040C20E94F6
:102F30009F1A009142031091430320914403309162
:102F40004503601B710B820B930B693E7340810537
:102F5000910508F42CC20E949F1A6093420370935B
:102F6000430380934403909345030E94AA0F1FC21A
:102F70000E94AB1A6B017C018091FA038430D1F47A
:102F80008FE70E94630406EF12E0E091DD03E77033
:102F9000F0E0EC56FD4F808190E09801265F3240D2
:102FA000281739070CF053CE0E947604D8018D9370
:102FB0008D01EBCFE091DD03E770F0E0EC56FD4FC3
:102FC00040814F5F21E0BE016F5F7F4F80E20E9432
:102FD000540A882371F0109346030E949F1A60934D
:102FE000420370934303809344039093450390E01E
:102FF00026CEE091DD03E770F0E0EC56FD4F408116
:1030000050E0BE016E5F7F4F86EF92E00E941B2072
:1030100025CE882309F46CCE1092400369CE982FF8
:103020009873983309F064CE9091ED02892787FF59
:103030005FCE90589093ED028091E503853209F0C0
:1030400057CE10E0212F30E08091F602877090E09B
:10305000821793070CF44CCE1F5FE12FF0E0EA508B
:10306000FD4F608188E094E00E94931DEBCF80913A
:10307000ED029091F602982796FD5AC0807C90E46C
:1030800089278093ED028091CC023091CB02831787
:10309000D1F0EEEEF2E020E02F5F90E0DC01A353F0
:1030A000BD4F4C91419301968F719927283011F0B3
:1030B0008313F2CF8093CC02295C8091ED02282B00
:1030C0002093ED0235C0809174038093EE028091CD
:1030D000E203863251F482E10E94F81B95958795B0
:1030E000959587958093EF0202C01092EF02809130
:1030F000E303863251F483E10E94F81B959587958E
:10310000959587958093F00202C01092F00280910D
:103110007003909171039093F1028093F202809179
:103120006E0390916F039F770E9416048093F302C1
:1031300069E08DEE92E00E9492060E9401078111E3
:10314000E9CD0E946513F9CF80916E0390916F03D2
:10315000880F991F90936F0380936E0381E0809393
:103160004103111110C0C0927C03D0927D03E09204
:103170007E03F0927F0310927803109279031092ED
:103180007A0310927B031F5F1093470385EB93E054
:103190000E94D202640D751D861D971D60938403E5
:1031A0007093850380938603909387032D9A81E023
:1031B0000E94ED0D0E944C0C03C0101709F4A6C02C
:1031C00080914703882309F478CE8091F603882301
:1031D000D9F090916903911117C040917C035091EF
:1031E0007D0360917E0370917F0346015701841A2D
:1031F000950AA60AB70A90E00E943602681579057A
:103200008A059B0508F4B4C08091F8038823D9F09F
:1032100090916B03911117C040917C0350917D03F5
:1032200060917E0370917F0346015701841A950ACD
:10323000A60AB70A90E00E943602681579058A0549
:103240009B0508F4ACC08091F7038823D9F09091D6
:103250006A03911117C040917C0350917D036091E6
:103260007E0370917F0346015701841A950AA60ACE
:10327000B70A90E00E943602681579058A059B0519
:1032800008F491C08091EE039091EF03A091F003B8
:10329000B091F103892B8A2B8B2B09F40ECE8091F0
:1032A000780390917903A0917A03B0917B03009702
:1032B000A105B10509F401CEC81AD90AEA0AFB0A28
:1032C000F7FCFBCD2091F30330E0A8EEB3E00E94C1
:1032D0004B1F6C157D058E059F0508F0EECD809186
:1032E000EC03829581700E946A0780E00E947C0551
:1032F0000E9457060E949F1A616060937803709342
:10330000790380937A0390937B03D7CD80918403D4
:1033100090918503A0918603B09187032401350124
:10332000481A590A6A0A7B0A85EB93E00E94D20286
:103330009B01AC01A12FB0E00E945A1F64157505D6
:103340008605970508F03CCF10926F0310926E032C
:1033500081E080934103109273030E944C0C809291
:10336000840390928503A0928603B092870328CFAE
:1033700081E0809369030E94C10C8091F2030E9456
:103380005B026C0D7D1D8E1D9F1D61606093780337
:103390007093790380937A0390937B0335CF81E018
:1033A00080936B0350CF81E080936A036BCF6A9662
:1033B000E0E10C94FC1F8230E8F4E82FF0E0EE0F1F
:1033C000FF1FE550FC4F71836083813041F0809195
:1033D00069008C7F842B80936900E89A089580911E
:1033E0006900440F551F440F551F837F842B809322
:1033F0006900E99A08951F920F920FB60F92112457
:103400002F933F934F935F936F937F938F939F93EC
:10341000AF93BF93EF93FF938091FB039091FC03D5
:10342000892B29F0E091FB03F091FC030995FF91B2
:10343000EF91BF91AF919F918F917F916F915F912C
:103440004F913F912F910F900FBE0F901F901895A5
:103450001F920F920FB60F9211242F933F934F9309
:103460005F936F937F938F939F93AF93BF93EF93EC
:10347000FF938091FD039091FE03892B29F0E09149
:10348000FD03F091FE030995FF91EF91BF91AF917C
:103490009F918F917F916F915F914F913F912F916C
:1034A0000F900FBE0F901F9018951F920F920FB69E
:1034B0000F9211242F933F938F939F93AF93BF93BA
:1034C0008091000490910104A0910204B091030442
:1034D0003091FF0323E0230F2D3720F40196A11D27
:1034E000B11D05C026E8230F0296A11DB11D209332
:1034F000FF038093000490930104A0930204B0930F
:1035000003048091040490910504A0910604B091F5
:1035100007040196A11DB11D809304049093050436
:10352000A0930604B0930704BF91AF919F918F9130
:103530003F912F910F900FBE0F901F9018952FB7AE
:10354000F8946091000470910104809102049091BC
:1035500003042FBF08953FB7F8948091040490911D
:103560000504A0910604B091070426B5A89B05C0E8
:103570002F3F19F00196A11DB11D3FBF6627782F7F
:10358000892F9A2F620F711D811D911D42E0660FD8
:10359000771F881F991F4A95D1F70895CF92DF9220
:1035A000EF92FF92CF93DF936B017C010E94AB1AE5
:1035B000EB01C114D104E104F10479F00E94AB1ACB
:1035C0006C1B7D0B683E7340A0F381E0C81AD108E4
:1035D000E108F108C851DC4FECCFDF91CF91FF90AB
:1035E000EF90DF90CF9008950197009739F0880F02
:1035F000991F880F991F02970197F1F70895789402
:1036000084B5826084BD84B5816084BD85B58260E7
:1036100085BD85B5816085BDEEE6F0E08081816085
:103620008083E1E8F0E01082808182608083808185
:1036300081608083E0E8F0E0808181608083E1EB5D
:10364000F0E0808184608083E0EBF0E08081816045
:103650008083EAE7F0E080818460808380818260FB
:1036600080838081816080838081806880831092E4
:10367000C1000895833081F028F4813099F08230C0
:10368000A1F008958630A9F08730B9F08430D1F4E4
:10369000809180008F7D03C0809180008F77809320
:1036A0008000089584B58F7702C084B58F7D84BD76
:1036B00008958091B0008F7703C08091B0008F7D16
:1036C0008093B0000895CF93DF9390E0FC01E4581D
:1036D000FF4F2491FC01E057FF4F8491882349F16B
:1036E00090E0880F991FFC01E854FF4FA591B49119
:1036F00082559F4FFC01C591D4919FB7611108C0BD
:10370000F8948C91209582238C93888182230AC01F
:10371000623051F4F8948C91322F309583238C933E
:103720008881822B888304C0F8948C91822B8C939F
:103730009FBFDF91CF910895A1E0B0E0E2EAFBE105
:103740000C94EC1F282F30E0F901E859FF4F8491C9
:10375000F901E458FF4F1491F901E057FF4F04912C
:103760000023C9F0882321F069830E943A1B6981F4
:10377000E02FF0E0EE0FFF1FE255FF4FA591B4914F
:103780009FB7F8948C91611103C01095812301C0FB
:10379000812B8C939FBF2196E4E00C940820CF935B
:1037A000DF93282F30E0F901E859FF4F8491F901A8
:1037B000E458FF4FD491F901E057FF4FC491CC2357
:1037C00091F081110E943A1BEC2FF0E0EE0FFF1FE9
:1037D000EC55FF4FA591B4912C912D2381E090E001
:1037E00021F480E002C080E090E0DF91CF91089565
:1037F0008E3008F08E5087702091B70190E4299F99
:1038000090011124822B80937C0080917A00806447
:1038100080937A0080917A0086FDFCCF80917800B9
:103820002091790090E0922B0895A0E0B0E0EBE1C8
:10383000FCE10C94E81F6C017A01EB01E60EF71E27
:1038400000E010E0CE15DF0561F06991D601ED9141
:10385000FC910190F081E02DC6010995080F191F18
:10386000F1CFC801CDB7DEB7E8E00C9404206115B4
:10387000710589F0DB010D900020E9F7AD014150A1
:103880005109461B570BDC01ED91FC910280F3813D
:10389000E02D0995089580E090E008950E94371C7E
:1038A0000895DC01ED91FC910190F081E02D0995E6
:1038B00008950F931F93CF93DF93EC016DE00E9467
:1038C000511C8C016AE0CE010E94511C800F911F97
:1038D000DF91CF911F910F9108950F931F93CF9375
:1038E000DF93EC010E94371C8C01CE010E94591C11
:1038F000800F911FDF91CF911F910F9108950F932A
:103900001F93CF93DF93EC010E94511C8C01CE01D9
:103910000E94591C800F911FDF91CF911F910F9131
:103920000895A1E2B0E0E7E9FCE10C94E41F7C011A
:10393000C42EE52FCB01D22E19A221E02D1510F0B7
:103940002AE0D22E8E010F5D1F4F8D2C912CA12CC1
:10395000B12C6C2D7E2FA50194010E949D1F8C2DF2
:10396000D29E80191124015011098A3010F4805D13
:1039700001C0895CF801808321153105410551059D
:1039800021F0C22EE32FCA01E4CFB801C7010E9483
:10399000371CA196ECE00C940020A0E0B0E0E3ED31
:1039A000FCE10C94E81FEC016A017B012115310553
:1039B00041F4E881F9810190F081E02D642F0995AF
:1039C0001DC02A303105A9F477FF12C06DE20E94B4
:1039D000511C8C0144275527BA014C195D096E0909
:1039E0007F092AE0CE010E94911C800F911F06C022
:1039F0002AE0B701A601CE010E94911CCDB7DEB727
:103A0000E8E00C9404200F931F93CF93DF93EC0115
:103A10009A01AB01662757FD6095762F0E94CD1C59
:103A20008C01CE010E94591C800F911FDF91CF9114
:103A30001F910F9108952115310549F4DC01ED9195
:103A4000FC910190F081E02D642F099508950E946A
:103A5000911C08959A01462F50E060E070E00E94AA
:103A60001B1D08959A01AB0160E070E00E941B1DD0
:103A70000895FC0124853585F901E05CFF4F8081C4
:103A80009181F901EE5BFF4F20813181821B930B05
:103A90008F7399270895FC0184859585FC01E05C6E
:103AA000FF4F40815181FC01EE5BFF4F208131814E
:103AB0004217530741F00190F081E02DE80FF91F04
:103AC000808190E008958FEF9FEF0895FC01848539
:103AD0009585FC01E05CFF4F40815181FC01EE5B6C
:103AE000FF4F208131814217530779F0A081B181C6
:103AF000A80FB91F8C91208131812F5F3F4F2F7309
:103B000033273183208390E008958FEF9FEF08954E
:103B1000FC0181A1882329F0A489B5898C9186FFB5
:103B2000FBCF11A20895CF93DF93FC012685378543
:103B3000D901A05CBF4F8D919C91119701968F7315
:103B40009927E901CE5BDF4F48815981841795079A
:103B5000D9F30D90BC91A02DA20FB31F6C93A68535
:103B6000B785A05CBF4F11969C938E93A689B789A9
:103B70002C9181E090E0078C02C0880F991F0A9475
:103B8000E2F7282B2C9381E081A30488F589E02DAE
:103B900080818064808381E090E0DF91CF910895FF
:103BA00008951F920F920FB60F9211242F933F93F7
:103BB0004F938F939F93EF93FF938091C00082FD6B
:103BC0001CC04091C6008091AE049091AF04019654
:103BD0008F7399272091B0043091B1048217930715
:103BE00071F0E091AE04F091AF04E259FB4F4083D5
:103BF0009093AF048093AE0402C08091C600FF9101
:103C0000EF919F918F914F913F912F910F900FBE08
:103C10000F901F90189588E094E00E94391D892B21
:103C200011F00E94D01D08951F920F920FB60F92AF
:103C300011242F933F938F939F93EF93FF932091A2
:103C40006A0430916B0480916C0490916D04281784
:103C5000390731F48091C1008F7D8093C10014C079
:103C6000E0916C04F0916D04E65DFB4F2081809142
:103C70006C0490916D0401968F73992790936D0455
:103C800080936C042093C600FF91EF919F918F91D8
:103C90003F912F910F900FBE0F901F901895A0E0AD
:103CA000B0E0E5E5FEE10C94E41FFC011382128212
:103CB00088EE93E0A0E0B0E084839583A683B78389
:103CC0008CEB92E091838083758764875787468762
:103CD000318B208B138B028BF58AE48AD78AC68AB4
:103CE000B18EA08E938E828E8F85848F8889858FEA
:103CF0008989868F8A89878F8B8980A3ECE00C94D1
:103D00000020CF92DF92EF92FF92CF93DF93EC01EE
:103D10006A017B01411581EE580761057105F9F0D3
:103D2000EC89FD8981E090E008A002C0880F991F0E
:103D30000A94E2F7808360E079E08DE390E0A701E8
:103D400096010E949D1F2150310941095109569544
:103D5000479537952795211580E1380798F0EC892C
:103D6000FD89108260E874E88EE190E0A701960179
:103D70000E949D1F215031094109510956954795CF
:103D800037952795E889F9893083EA89FB8920836B
:103D900019A2EE89FF89408181E090E09C010C8CA2
:103DA00002C0220F331F0A94E2F7422B4083EE89B0
:103DB000FF8940819C010D8C02C0220F331F0A94A1
:103DC000E2F7422B4083EE89FF8940819C010E8CF3
:103DD00002C0220F331F0A94E2F7422B4083EE8980
:103DE000FF8920810F8C02C0880F991F0A94E2F787
:103DF000809582238083DF91CF91FF90EF90DF90B9
:103E0000CF9008958F929F92AF92BF92CF92DF9200
:103E1000EF92FF920F931F9381E08F9385E08F9332
:103E200087E08F9383E08F9384E08F93E6EC8E2E70
:103E3000912CF2ECAF2EB12CA1ECCA2ED12CB0EC0F
:103E4000EB2EF12C04EC10E025EC30E04AE254E0DB
:103E50006EE674E088E094E00E944F1E0F900F9091
:103E60000F900F900F901F910F91FF90EF90DF90A8
:103E7000CF90BF90AF909F908F9008950E94FF1AAF
:103E80000E940612CBE0DEE10E94FC152097E1F3D0
:103E90000E940B1EF9CFA29FB001B39FC001A39F48
:103EA000700D811D1124911DB29F700D811D112473
:103EB000911D08950E944B1FA59F900DB49F900DDA
:103EC000A49F800D911D11240895B7FF0C945A1FD3
:103ED0000E945A1F821B930B0895DB018F939F93BF
:103EE0000E945A1FBF91AF91A29F800D911DA39F69
:103EF000900DB29F900D11240895991B79E004C094
:103F0000991F961708F0961B881F7A95C9F7809518
:103F10000895AA1BBB1B51E107C0AA1FBB1FA61710
:103F2000B70710F0A61BB70B881F991F5A95A9F762
:103F300080959095BC01CD010895A1E21A2EAA1B8F
:103F4000BB1BFD010DC0AA1FBB1FEE1FFF1FA21749
:103F5000B307E407F50720F0A21BB30BE40BF50B46
:103F6000661F771F881F991F1A9469F760957095CF
:103F7000809590959B01AC01BD01CF010895052E60
:103F800097FB1EF400940E94D61F57FD07D00E9495
:103F90009D1F07FC03D04EF40C94D61F50954095FE
:103FA000309521953F4F4F4F5F4F089590958095E5
:103FB000709561957F4F8F4F9F4F08952F923F923D
:103FC0004F925F926F927F928F929F92AF92BF9229
:103FD000CF92DF92EF92FF920F931F93CF93DF93D5
:103FE000CDB7DEB7CA1BDB0B0FB6F894DEBF0FBE32
:103FF000CDBF09942A88398848885F846E847D847F
:104000008C849B84AA84B984C884DF80EE80FD8080
:104010000C811B81AA81B981CE0FD11D0FB6F894F6
:10402000DEBF0FBECDBFED010895EE0FFF1F05905F
:10403000F491E02D0994FB01DC0102C001900D9286
:1040400041505040D8F70895F999FECF92BD81BDF7
:10405000F89A992780B50895262FF999FECF1FBAAF
:1040600092BD81BD20BD0FB6F894FA9AF99A0FBEA1
:0840700001960895F894FFCFBA
:104078000000B204200008409C88130002000200DF
:104088000200020002000200020002000200020018
:104098000200020002000200020002802500000562
:1040A800400AA1204EA50020244EA52C2330C01282
:1040B80000001A400AA1204EA5001B1E27522C23DF
:1040C800308025000005400AA1204EA50020244E7E
:1040D800A52C2330004B000006400AD0009D490063
:1040E8007B289D492C233000E1000005400A45014A
:1040F800D7DC03B81E0EBF00232E48E801008A4013
:104108000A6001555502AD1E20000023C800200199
:10411800270121022B032203260423042605240653
:104128002506280629062A0154582074696D656FEA
:104138007574210057616974696E672062696E64DD
:104148000A00476F7420706B740A00646174612000
:10415800676F6F640A007363616E6E6572206D6FBE
:104168006465004F70656E4C52536E67205258203C
:104178007374617274696E672000206F6E204857EF
:10418800200053617665642062696E6420646174FE
:104198006120746F20454550524F4D0A00492061F7
:1041A8006D20736C61766500456E746572696E6723
:1041B800206E6F726D616C206D6F646500454550AF
:1041C800524F4D2064617461206E6F742076616C6B
:1041D8006964206F722062696E64206A756D707000
:1041E8006572207365742C20666F7263696E672030
:1041F80062696E640A0052582068616E6700B200F6
:10420800F4014C0300070B0C101115000A030E12E1
:104218001300010400000000080001000010000065
:10422800200000000100000200000000931D151C82
:08423800391D661D4B1D881D98
:00000001FF
